BL51 BANKED LINKER/LOCATER V6.22                                                        11/20/2017  11:41:10  PAGE 1


BL51 BANKED LINKER/LOCATER V6.22, INVOKED BY:
C:\KEIL4\C51\BIN\BL51.EXE .\OBJ\MAIN.obj TO .\OBJ\5D_TWI0_S_P22P24 PRINT (.\LST\5D_TWI0_S_P22P24.m51) RAMSIZE (256)


MEMORY MODEL: SMALL


INPUT MODULES INCLUDED:
  .\OBJ\MAIN.obj (MAIN)
  C:\KEIL4\C51\LIB\C51S.LIB (?C_STARTUP)
  C:\KEIL4\C51\LIB\C51S.LIB (?C?CLDPTR)
  C:\KEIL4\C51\LIB\C51S.LIB (?C?CCASE)
  C:\KEIL4\C51\LIB\C51S.LIB (?C_INIT)


LINK MAP OF MODULE:  .\OBJ\5D_TWI0_S_P22P24 (MAIN)


            TYPE    BASE      LENGTH    RELOCATION   SEGMENT NAME
            -----------------------------------------------------

            * * * * * * *   D A T A   M E M O R Y   * * * * * * *
            REG     0000H     0008H     ABSOLUTE     "REG BANK 0"
            DATA    0008H     0005H     UNIT         ?DT?MAIN
                    000DH     0013H                  *** GAP ***
            BIT     0020H.0   0000H.2   UNIT         ?BI?MAIN
                    0020H.2   0000H.6                *** GAP ***
            IDATA   0021H     0001H     UNIT         ?STACK

            * * * * * * *  X D A T A   M E M O R Y  * * * * * * *
            XDATA   0000H     0010H     UNIT         ?XD?MAIN

            * * * * * * *   C O D E   M E M O R Y   * * * * * * *
            CODE    0000H     0003H     ABSOLUTE     
                    0003H     0008H                  *** GAP ***
            CODE    000BH     0003H     ABSOLUTE     
            CODE    000EH     003FH     UNIT         ?PR?INITSYSTEM?MAIN
            CODE    004DH     0014H     UNIT         ?C_INITSEG
                    0061H     0002H                  *** GAP ***
            CODE    0063H     0003H     ABSOLUTE     
            CODE    0066H     008CH     UNIT         ?C_C51STARTUP
            CODE    00F2H     0081H     UNIT         ?PR?INT_TWSI?MAIN
            CODE    0173H     003FH     UNIT         ?C?LIB_CODE
            CODE    01B2H     002CH     UNIT         ?PR?_SENDHEX?MAIN
            CODE    01DEH     002BH     UNIT         ?PR?MAIN?MAIN
            CODE    0209H     0027H     UNIT         ?PR?INT_T0?MAIN
            CODE    0230H     0013H     UNIT         ?PR?_SENDSTR?MAIN
            CODE    0243H     0013H     UNIT         ?PR?RESTARTTWI0?MAIN
            CODE    0256H     0012H     UNIT         ?PR?_SENDBYTE?MAIN
            CODE    0268H     000BH     UNIT         ?PR?_DELAYMS?MAIN



OVERLAY MAP OF MODULE:   .\OBJ\5D_TWI0_S_P22P24 (MAIN)


SEGMENT
  +--> CALLED SEGMENT
BL51 BANKED LINKER/LOCATER V6.22                                                      11/20/2017  11:41:10  PAGE 2


---------------------
?C_C51STARTUP
  +--> ?PR?MAIN?MAIN
  +--> ?C_INITSEG

?PR?MAIN?MAIN
  +--> ?PR?INITSYSTEM?MAIN
  +--> ?PR?_DELAYMS?MAIN
  +--> ?PR?RESTARTTWI0?MAIN



SYMBOL TABLE OF MODULE:  .\OBJ\5D_TWI0_S_P22P24 (MAIN)

  VALUE           TYPE          NAME
  ----------------------------------

  -------         MODULE        MAIN
  C:0000H         SYMBOL        _ICE_DUMMY_
  D:0095H         PUBLIC        P2M0
  D:0092H         PUBLIC        P2M1
  D:0090H         PUBLIC        P1
  D:00A0H         PUBLIC        P2
  D:00C0H         PUBLIC        XICON
  D:00B0H         PUBLIC        P3
  D:00E8H         PUBLIC        P4
  D:00ADH         PUBLIC        EIE1
  D:00F8H         PUBLIC        P6
  D:00D3H         PUBLIC        SISTA
  D:00ACH         PUBLIC        SFRPI
  B:00A8H.7       PUBLIC        EA
  D:00A8H         PUBLIC        IE
  C:00F2H         PUBLIC        INT_TWSI
  D:00B8H         PUBLIC        IP0L
  D:0093H         PUBLIC        T2MOD1
  D:0008H         PUBLIC        BufAddr
  D:0009H         PUBLIC        TWI0Ovtime
  C:000EH         PUBLIC        InitSystem
  D:00C7H         PUBLIC        CKCON0
  D:000BH         PUBLIC        delayNmS
  C:0256H         PUBLIC        _SendByte
  D:00D8H         PUBLIC        CCON
  C:01DEH         PUBLIC        main
  B:00C8H.5       PUBLIC        RCLK_TF2L
  B:0020H.0       PUBLIC        bES0
  C:01B2H         PUBLIC        _SendHex
  C:0268H         PUBLIC        _DelayMs
  B:00A0H.2       PUBLIC        P22
  D:0089H         PUBLIC        TMOD
  D:0088H         PUBLIC        TCON
  B:00B0H.5       PUBLIC        P35
  B:0020H.1       PUBLIC        bAddrorData
  X:0000H         PUBLIC        TestBuf
  C:0230H         PUBLIC        _SendStr
  B:00A8H.4       PUBLIC        ES0
  B:00A8H.1       PUBLIC        ET0
  D:008CH         PUBLIC        TH0
BL51 BANKED LINKER/LOCATER V6.22                                                      11/20/2017  11:41:10  PAGE 3


  B:0098H.1       PUBLIC        TI0
  D:008DH         PUBLIC        TH1
  C:0209H         PUBLIC        INT_T0
  D:008AH         PUBLIC        TL0
  B:0088H.4       PUBLIC        TR0
  B:0088H.6       PUBLIC        TR1
  D:0099H         PUBLIC        S0BUF
  D:0087H         PUBLIC        PCON0
  D:0098H         PUBLIC        S0CON
  D:00C8H         PUBLIC        T2CON
  C:0243H         PUBLIC        ReStartTWI0
  B:00C8H.4       PUBLIC        TCLK_TL2IE
  D:00A3H         PUBLIC        AUXR2
  D:00D1H         PUBLIC        SIADR
  D:00A4H         PUBLIC        AUXR3
  D:00D2H         PUBLIC        SIDAT
  D:00D0H         PUBLIC        PSW
  D:00D4H         PUBLIC        SICON
  -------         PROC          INT_T0
  C:0209H         LINE#         52
  C:020BH         LINE#         54
  C:020EH         LINE#         55
  C:0211H         LINE#         57
  C:021FH         LINE#         58
  C:022DH         LINE#         60
  -------         ENDPROC       INT_T0
  -------         PROC          _SENDBYTE
  D:0007H         SYMBOL        tByte
  C:0256H         LINE#         63
  C:0256H         LINE#         64
  C:0256H         LINE#         65
  C:025AH         LINE#         66
  C:025CH         LINE#         67
  C:025EH         LINE#         68
  C:0261H         LINE#         69
  C:0263H         LINE#         70
  C:0267H         LINE#         71
  -------         ENDPROC       _SENDBYTE
  -------         PROC          _SENDSTR
  D:0001H         SYMBOL        PStr
  C:0230H         LINE#         75
  C:0230H         LINE#         76
  C:0230H         LINE#         77
  C:0236H         LINE#         78
  C:0236H         LINE#         79
  C:0239H         LINE#         80
  C:0240H         LINE#         81
  C:0242H         LINE#         82
  -------         ENDPROC       _SENDSTR
  -------         PROC          _SENDHEX
  D:0006H         SYMBOL        ToSend
  -------         DO            
  D:0005H         SYMBOL        x
  -------         ENDDO         
  C:01B2H         LINE#         84
  C:01B4H         LINE#         85
  C:01B4H         LINE#         87
BL51 BANKED LINKER/LOCATER V6.22                                                      11/20/2017  11:41:10  PAGE 4


  C:01B9H         LINE#         88
  C:01BFH         LINE#         89
  C:01BFH         LINE#         90
  C:01C1H         LINE#         91
  C:01C3H         LINE#         93
  C:01C3H         LINE#         94
  C:01C9H         LINE#         95
  C:01C9H         LINE#         96
  C:01CDH         LINE#         97
  C:01D3H         LINE#         98
  C:01D3H         LINE#         99
  C:01D5H         LINE#         100
  C:01D7H         LINE#         102
  C:01D7H         LINE#         103
  C:01DDH         LINE#         104
  C:01DDH         LINE#         105
  -------         ENDPROC       _SENDHEX
  -------         PROC          INT_TWSI
  C:00F2H         LINE#         107
  C:0101H         LINE#         109
  C:0103H         LINE#         110
  C:0106H         LINE#         111
  C:012BH         LINE#         112
  C:012BH         LINE#         113
  C:012BH         LINE#         114
  C:012BH         LINE#         119
  C:012BH         LINE#         120
  C:012EH         LINE#         121
  C:012EH         LINE#         122
  C:012EH         LINE#         123
  C:0130H         LINE#         125
  C:0130H         LINE#         129
  C:0130H         LINE#         130
  C:0130H         LINE#         132
  C:0133H         LINE#         133
  C:0136H         LINE#         134
  C:013BH         LINE#         135
  C:013DH         LINE#         137
  C:013DH         LINE#         138
  C:013DH         LINE#         139
  C:0140H         LINE#         140
  C:0143H         LINE#         141
  C:0149H         LINE#         142
  C:014BH         LINE#         143
  C:014BH         LINE#         144
  C:014BH         LINE#         145
  C:014BH         LINE#         146
  C:014BH         LINE#         147
  C:014EH         LINE#         149
  C:0151H         LINE#         150
  C:0151H         LINE#         151
  C:0151H         LINE#         152
  C:0153H         LINE#         153
  C:0156H         LINE#         155
  C:0157H         LINE#         156
  C:0158H         LINE#         157
  C:0159H         LINE#         158
BL51 BANKED LINKER/LOCATER V6.22                                                      11/20/2017  11:41:10  PAGE 5


  C:015AH         LINE#         159
  C:015BH         LINE#         160
  C:015CH         LINE#         161
  C:015DH         LINE#         162
  C:015EH         LINE#         163
  C:015FH         LINE#         164
  C:0160H         LINE#         165
  C:0161H         LINE#         166
  C:0162H         LINE#         168
  C:0164H         LINE#         170
  C:0166H         LINE#         171
  -------         ENDPROC       INT_TWSI
  -------         PROC          RESTARTTWI0
  C:0243H         LINE#         180
  C:0243H         LINE#         181
  C:0243H         LINE#         182
  C:0246H         LINE#         183
  C:0249H         LINE#         184
  C:024CH         LINE#         185
  C:024DH         LINE#         186
  C:024EH         LINE#         187
  C:024FH         LINE#         188
  C:0252H         LINE#         189
  C:0255H         LINE#         190
  -------         ENDPROC       RESTARTTWI0
  -------         PROC          INITSYSTEM
  C:000EH         LINE#         194
  C:000EH         LINE#         195
  C:000EH         LINE#         196
  C:0011H         LINE#         199
  C:0014H         LINE#         201
  C:0017H         LINE#         202
  C:001AH         LINE#         203
  C:001CH         LINE#         207
  C:001FH         LINE#         209
  C:0022H         LINE#         211
  C:0025H         LINE#         212
  C:0027H         LINE#         213
  C:0029H         LINE#         215
  C:002CH         LINE#         216
  C:002FH         LINE#         218
  C:0031H         LINE#         221
  C:0039H         LINE#         223
  C:003CH         LINE#         224
  C:003FH         LINE#         227
  C:0042H         LINE#         228
  C:0045H         LINE#         230
  C:0048H         LINE#         231
  C:004AH         LINE#         233
  C:004CH         LINE#         235
  -------         ENDPROC       INITSYSTEM
  -------         PROC          MAIN
  C:01DEH         LINE#         237
  C:01DEH         LINE#         238
  C:01DEH         LINE#         239
  C:01E1H         LINE#         240
  C:01E3H         LINE#         241
BL51 BANKED LINKER/LOCATER V6.22                                                      11/20/2017  11:41:10  PAGE 6


  C:01EAH         LINE#         242
  C:01ECH         LINE#         244
  C:01ECH         LINE#         245
  C:01ECH         LINE#         246
  C:01F2H         LINE#         247
  C:01F2H         LINE#         248
  C:01F7H         LINE#         249
  C:01F9H         LINE#         250
  C:01F9H         LINE#         253
  C:01FFH         LINE#         254
  C:01FFH         LINE#         256
  C:0204H         LINE#         257
  C:0207H         LINE#         258
  C:0207H         LINE#         259
  -------         ENDPROC       MAIN
  -------         PROC          _DELAYMS
  D:0006H         SYMBOL        DelayTime
  C:0268H         LINE#         263
  C:0268H         LINE#         264
  C:0268H         LINE#         265
  C:026CH         LINE#         266
  C:0272H         LINE#         267
  C:0272H         LINE#         269
  C:0272H         LINE#         270
  -------         ENDPROC       _DELAYMS
  -------         ENDMOD        MAIN

  -------         MODULE        ?C?CLDPTR
  C:0173H         PUBLIC        ?C?CLDPTR
  -------         ENDMOD        ?C?CLDPTR

  -------         MODULE        ?C?CCASE
  C:018CH         PUBLIC        ?C?CCASE
  -------         ENDMOD        ?C?CCASE

*** WARNING L16: UNCALLED SEGMENT, IGNORED FOR OVERLAY PROCESS
    SEGMENT: ?PR?_SENDSTR?MAIN

*** WARNING L16: UNCALLED SEGMENT, IGNORED FOR OVERLAY PROCESS
    SEGMENT: ?PR?_SENDHEX?MAIN

Program Size: data=14.2 xdata=16 code=617
LINK/LOCATE RUN COMPLETE.  2 WARNING(S),  0 ERROR(S)
